 SetNativeMethodPrefix002

 Timestamp is e793eba0 (reproducible build file hash)

 Preferred load address is 0000000180000000

 Start         Length     Name                   Class
 0001:00000000 000031b0H .text$mn                CODE
 0001:000031b0 00000036H .text$mn$00             CODE
 0001:000031e6 00000092H .text$x                 CODE
 0002:00000000 000001c8H .idata$5                DATA
 0002:000001c8 00000038H .00cfg                  DATA
 0002:00000200 00000008H .CRT$XCA                DATA
 0002:00000208 00000008H .CRT$XCZ                DATA
 0002:00000210 00000008H .CRT$XIA                DATA
 0002:00000218 00000008H .CRT$XIC                DATA
 0002:00000220 00000008H .CRT$XIZ                DATA
 0002:00000228 00000008H .CRT$XLA                DATA
 0002:00000230 00000008H .CRT$XLZ                DATA
 0002:00000238 00000008H .CRT$XPA                DATA
 0002:00000240 00000008H .CRT$XPZ                DATA
 0002:00000248 00000008H .CRT$XTA                DATA
 0002:00000250 00000010H .CRT$XTZ                DATA
 0002:00000258 00000000H .gehcont$y              DATA
 0002:00000258 00000000H .gfids$y                DATA
 0002:00000260 00001ea0H .rdata                  DATA
 0002:00002100 00000000H .rdata$CastGuardVftablesA DATA
 0002:00002100 00000000H .rdata$CastGuardVftablesC DATA
 0002:00002100 00000028H .rdata$T                DATA
 0002:00002128 000000b8H .rdata$voltmd           DATA
 0002:000021e0 00000328H .rdata$zzzdbg           DATA
 0002:00002508 00000008H .rtc$IAA                DATA
 0002:00002510 00000008H .rtc$IZZ                DATA
 0002:00002518 00000008H .rtc$TAA                DATA
 0002:00002520 00000008H .rtc$TZZ                DATA
 0002:00002528 00000004H .tls                    DATA
 0002:0000252c 00000004H .tls$                   DATA
 0002:00002530 00000008H .tls$ZZZ                DATA
 0002:00002538 00000338H .xdata                  DATA
 0002:00002870 000003bcH .edata                  DATA
 0002:00002c2c 0000008cH .idata$2                DATA
 0002:00002cb8 00000018H .idata$3                DATA
 0002:00002cd0 000001c8H .idata$4                DATA
 0002:00002e98 00000486H .idata$6                DATA
 0003:00000000 00000080H .data                   DATA
 0003:00000080 0001b238H .bss                    DATA
 0004:00000000 000003b4H .pdata                  DATA

  Address         Publics by Value              Rva+Base               Lib:Object

 0000:00000000       __AbsoluteZero             0000000000000000     <absolute>
 0000:00000000       ___safe_se_handler_count   0000000000000000     <absolute>
 0000:00000000       ___safe_se_handler_table   0000000000000000     <absolute>
 0000:00000000       __arm64x_extra_rfe_table   0000000000000000     <absolute>
 0000:00000000       __arm64x_extra_rfe_table_size 0000000000000000     <absolute>
 0000:00000000       __arm64x_native_entrypoint 0000000000000000     <absolute>
 0000:00000000       __arm64x_redirection_metadata 0000000000000000     <absolute>
 0000:00000000       __arm64x_redirection_metadata_count 0000000000000000     <absolute>
 0000:00000000       __dynamic_value_reloc_table 0000000000000000     <absolute>
 0000:00000000       __enclave_config           0000000000000000     <absolute>
 0000:00000000       __guard_check_icall_a64n_fptr 0000000000000000     <absolute>
 0000:00000000       __guard_eh_cont_count      0000000000000000     <absolute>
 0000:00000000       __guard_eh_cont_table      0000000000000000     <absolute>
 0000:00000000       __guard_fids_count         0000000000000000     <absolute>
 0000:00000000       __guard_fids_table         0000000000000000     <absolute>
 0000:00000000       __guard_iat_count          0000000000000000     <absolute>
 0000:00000000       __guard_iat_table          0000000000000000     <absolute>
 0000:00000000       __guard_longjmp_count      0000000000000000     <absolute>
 0000:00000000       __guard_longjmp_table      0000000000000000     <absolute>
 0000:00000000       __hybrid_auxiliary_iat     0000000000000000     <absolute>
 0000:00000000       __hybrid_auxiliary_iat_copy 0000000000000000     <absolute>
 0000:00000000       __hybrid_code_map          0000000000000000     <absolute>
 0000:00000000       __hybrid_code_map_count    0000000000000000     <absolute>
 0000:00000000       __x64_code_ranges_to_entry_points 0000000000000000     <absolute>
 0000:00000000       __x64_code_ranges_to_entry_points_count 0000000000000000     <absolute>
 0000:00000100       __guard_flags              0000000000000100     <absolute>
 0000:00000000       __ImageBase                0000000180000000     <linker-defined>
 0001:00000000       ?NewObject@JNIEnv_@@QEAAPEAV_jobject@@PEAV_jclass@@PEAU_jmethodID@@ZZ 0000000180001000 f i libSetNativeMethodPrefix002.obj
 0001:00000024       ?TranslateError@@YAPEBDW4jvmtiError@@@Z 0000000180001024 f   libSetNativeMethodPrefix002.obj
 0001:000002dc       ?nsk_jni_check_exception@@YAHPEAUJNIEnv_@@QEBDH@Z 00000001800012dc f   libSetNativeMethodPrefix002.obj
 0001:00000420       ?nsk_jni_lverify@@YAHHPEAUJNIEnv_@@HQEBDH1ZZ 0000000180001420 f   libSetNativeMethodPrefix002.obj
 0001:000004c0       Agent_Initialize           00000001800014c0 f   libSetNativeMethodPrefix002.obj
 0001:00000734       Agent_OnAttach             0000000180001734 f   libSetNativeMethodPrefix002.obj
 0001:00000734       Agent_OnLoad               0000000180001734 f   libSetNativeMethodPrefix002.obj
 0001:0000073c       Java_nsk_jvmti_SetNativeMethodPrefix_SetNativeMethodPrefix002_foo 000000018000173c f   libSetNativeMethodPrefix002.obj
 0001:0000076c       Java_nsk_jvmti_unit_FollowReferences_FollowRefObjects_addRefToVerify 000000018000176c f   libSetNativeMethodPrefix002.obj
 0001:00000928       Java_nsk_jvmti_unit_FollowReferences_FollowRefObjects_getTag 0000000180001928 f   libSetNativeMethodPrefix002.obj
 0001:000009e4       Java_nsk_jvmti_unit_FollowReferences_FollowRefObjects_resetRefsToVerify 00000001800019e4 f   libSetNativeMethodPrefix002.obj
 0001:000009ec       Java_nsk_jvmti_unit_FollowReferences_FollowRefObjects_resetTags 00000001800019ec f   libSetNativeMethodPrefix002.obj
 0001:00000a30       Java_nsk_jvmti_unit_FollowReferences_FollowRefObjects_setTag 0000000180001a30 f   libSetNativeMethodPrefix002.obj
 0001:00000c7c       Java_nsk_share_jvmti_ArgumentHandler_getAgentOptionsString 0000000180001c7c f   libSetNativeMethodPrefix002.obj
 0001:00000d28       Java_nsk_share_jvmti_DebugeeClass_checkStatus 0000000180001d28 f   libSetNativeMethodPrefix002.obj
 0001:00000db0       Java_nsk_share_jvmti_DebugeeClass_resetAgentData 0000000180001db0 f   libSetNativeMethodPrefix002.obj
 0001:00000e10       Java_nsk_share_jvmti_RedefineAgent_agentStatus 0000000180001e10 f   libSetNativeMethodPrefix002.obj
 0001:00000e1c       Java_nsk_share_jvmti_RedefineAgent_isRedefined 0000000180001e1c f   libSetNativeMethodPrefix002.obj
 0001:00000e28       Java_nsk_share_jvmti_RedefineAgent_redefineAttempted 0000000180001e28 f   libSetNativeMethodPrefix002.obj
 0001:00000e34       MA_checkStatus             0000000180001e34 f   libSetNativeMethodPrefix002.obj
 0001:00000ed8       __local_stdio_printf_options 0000000180001ed8 f i libSetNativeMethodPrefix002.obj
 0001:0000126c       exitOnError                000000018000226c f   libSetNativeMethodPrefix002.obj
 0001:00001320       fprintf                    0000000180002320 f i libSetNativeMethodPrefix002.obj
 0001:00001364       nsk_complain               0000000180002364 f   libSetNativeMethodPrefix002.obj
 0001:00001390       nsk_jvmti_createJVMTIEnv   0000000180002390 f   libSetNativeMethodPrefix002.obj
 0001:000014c0       nsk_jvmti_findOptionIntValue 00000001800024c0 f   libSetNativeMethodPrefix002.obj
 0001:0000155c       nsk_jvmti_findOptionValue  000000018000255c f   libSetNativeMethodPrefix002.obj
 0001:000015d4       nsk_jvmti_lverify          00000001800025d4 f   libSetNativeMethodPrefix002.obj
 0001:000016c4       nsk_jvmti_parseOptions     00000001800026c4 f   libSetNativeMethodPrefix002.obj
 0001:00001914       nsk_jvmti_resetAgentData   0000000180002914 f   libSetNativeMethodPrefix002.obj
 0001:00001988       nsk_lcomplain              0000000180002988 f   libSetNativeMethodPrefix002.obj
 0001:000019a8       nsk_ldisplay               00000001800029a8 f   libSetNativeMethodPrefix002.obj
 0001:000019c8       nsk_ltrace                 00000001800029c8 f   libSetNativeMethodPrefix002.obj
 0001:000019e8       nsk_lvcomplain             00000001800029e8 f   libSetNativeMethodPrefix002.obj
 0001:00001ba0       nsk_lvdisplay              0000000180002ba0 f   libSetNativeMethodPrefix002.obj
 0001:00001bec       nsk_lverify                0000000180002bec f   libSetNativeMethodPrefix002.obj
 0001:00001c48       nsk_lvtrace                0000000180002c48 f   libSetNativeMethodPrefix002.obj
 0001:00001ca8       nsk_printf                 0000000180002ca8 f   libSetNativeMethodPrefix002.obj
 0001:00001cd0       nsk_vprintf                0000000180002cd0 f   libSetNativeMethodPrefix002.obj
 0001:00001d84       printf                     0000000180002d84 f i libSetNativeMethodPrefix002.obj
 0001:00002284       __raise_securityfailure    0000000180003284 f   MSVCRT:gs_report.obj
 0001:000022b8       __report_gsfailure         00000001800032b8 f   MSVCRT:gs_report.obj
 0001:000024f8       __GSHandlerCheck           00000001800034f8 f   MSVCRT:gshandler.obj
 0001:00002518       __GSHandlerCheckCommon     0000000180003518 f   MSVCRT:gshandler.obj
 0001:00002590       __security_check_cookie    0000000180003590 f   MSVCRT:amdsecgs.obj
 0001:000028d0       _DllMainCRTStartup         00000001800038d0 f   MSVCRT:dll_dllmain.obj
 0001:00002910       __scrt_acquire_startup_lock 0000000180003910 f   MSVCRT:utility.obj
 0001:0000294c       __scrt_dllmain_after_initialize_c 000000018000394c f   MSVCRT:utility.obj
 0001:00002980       __scrt_dllmain_before_initialize_c 0000000180003980 f   MSVCRT:utility.obj
 0001:00002998       __scrt_dllmain_crt_thread_attach 0000000180003998 f   MSVCRT:utility.obj
 0001:000029c0       __scrt_dllmain_crt_thread_detach 00000001800039c0 f   MSVCRT:utility.obj
 0001:000029d8       __scrt_dllmain_exception_filter 00000001800039d8 f   MSVCRT:utility.obj
 0001:00002a38       __scrt_dllmain_uninitialize_c 0000000180003a38 f   MSVCRT:utility.obj
 0001:00002a68       __scrt_dllmain_uninitialize_critical 0000000180003a68 f   MSVCRT:utility.obj
 0001:00002a7c       __scrt_initialize_crt      0000000180003a7c f   MSVCRT:utility.obj
 0001:00002ac8       __scrt_initialize_onexit_tables 0000000180003ac8 f   MSVCRT:utility.obj
 0001:00002b54       __scrt_is_nonwritable_in_current_image 0000000180003b54 f   MSVCRT:utility.obj
 0001:00002bec       __scrt_release_startup_lock 0000000180003bec f   MSVCRT:utility.obj
 0001:00002c10       __scrt_uninitialize_crt    0000000180003c10 f   MSVCRT:utility.obj
 0001:00002c3c       _onexit                    0000000180003c3c f   MSVCRT:utility.obj
 0001:00002c78       atexit                     0000000180003c78 f   MSVCRT:utility.obj
 0001:00002c90       __crt_debugger_hook        0000000180003c90 f   MSVCRT:utility_desktop.obj
 0001:00002c98       __scrt_fastfail            0000000180003c98 f   MSVCRT:utility_desktop.obj
 0001:00002de4       _guard_check_icall_nop     0000000180003de4 f i MSVCRT:guard_support.obj
 0001:00002de8       __security_init_cookie     0000000180003de8 f   MSVCRT:gs_support.obj
 0001:00002e94       DllMain                    0000000180003e94 f   MSVCRT:dll_dllmain_stub.obj
 0001:00002eb8       ?__scrt_initialize_type_info@@YAXXZ 0000000180003eb8 f   MSVCRT:tncleanup.obj
 0001:00002ec8       ?__scrt_uninitialize_type_info@@YAXXZ 0000000180003ec8 f   MSVCRT:tncleanup.obj
 0001:00002ed4       __local_stdio_scanf_options 0000000180003ed4 f i MSVCRT:default_local_stdio_options.obj
 0001:00002edc       __scrt_initialize_default_local_stdio_options 0000000180003edc f   MSVCRT:default_local_stdio_options.obj
 0001:00002ef8       __scrt_get_dyn_tls_init_callback 0000000180003ef8 f   MSVCRT:dyn_tls_init.obj
 0001:00002f00       _RTC_Initialize            0000000180003f00 f   MSVCRT:initsect.obj
 0001:00002f3c       _RTC_Terminate             0000000180003f3c f   MSVCRT:initsect.obj
 0001:00002f78       __isa_available_init       0000000180003f78 f   MSVCRT:cpu_disp.obj
 0001:00003124       _get_startup_argv_mode     0000000180004124 f   MSVCRT:argv_mode.obj
 0001:0000312c       __scrt_is_ucrt_dll_in_use  000000018000412c f   MSVCRT:ucrt_detection.obj
 0001:00003140       memcpy                     0000000180004140 f   vcruntime:VCRUNTIME140.dll
 0001:00003146       memset                     0000000180004146 f   vcruntime:VCRUNTIME140.dll
 0001:0000314c       strchr                     000000018000414c f   vcruntime:VCRUNTIME140.dll
 0001:00003152       __C_specific_handler       0000000180004152 f   vcruntime:VCRUNTIME140.dll
 0001:00003158       __std_type_info_destroy_list 0000000180004158 f   vcruntime:VCRUNTIME140.dll
 0001:0000315e       strcmp                     000000018000415e f   ucrt:api-ms-win-crt-string-l1-1-0.dll
 0001:00003164       strlen                     0000000180004164 f   ucrt:api-ms-win-crt-string-l1-1-0.dll
 0001:0000316a       _initterm                  000000018000416a f   ucrt:api-ms-win-crt-runtime-l1-1-0.dll
 0001:00003170       _initterm_e                0000000180004170 f   ucrt:api-ms-win-crt-runtime-l1-1-0.dll
 0001:00003176       _seh_filter_dll            0000000180004176 f   ucrt:api-ms-win-crt-runtime-l1-1-0.dll
 0001:0000317c       _configure_narrow_argv     000000018000417c f   ucrt:api-ms-win-crt-runtime-l1-1-0.dll
 0001:00003182       _initialize_narrow_environment 0000000180004182 f   ucrt:api-ms-win-crt-runtime-l1-1-0.dll
 0001:00003188       _initialize_onexit_table   0000000180004188 f   ucrt:api-ms-win-crt-runtime-l1-1-0.dll
 0001:0000318e       _register_onexit_function  000000018000418e f   ucrt:api-ms-win-crt-runtime-l1-1-0.dll
 0001:00003194       _execute_onexit_table      0000000180004194 f   ucrt:api-ms-win-crt-runtime-l1-1-0.dll
 0001:0000319a       _crt_atexit                000000018000419a f   ucrt:api-ms-win-crt-runtime-l1-1-0.dll
 0001:000031a0       _cexit                     00000001800041a0 f   ucrt:api-ms-win-crt-runtime-l1-1-0.dll
 0001:000031a8       __acrt_initialize          00000001800041a8 f   MSVCRT:ucrt_stubs.obj
 0001:000031a8       __acrt_thread_attach       00000001800041a8 f   MSVCRT:ucrt_stubs.obj
 0001:000031a8       __acrt_thread_detach       00000001800041a8 f   MSVCRT:ucrt_stubs.obj
 0001:000031a8       __acrt_uninitialize        00000001800041a8 f   MSVCRT:ucrt_stubs.obj
 0001:000031a8       __acrt_uninitialize_critical 00000001800041a8 f   MSVCRT:ucrt_stubs.obj
 0001:000031a8       __scrt_stub_for_acrt_initialize 00000001800041a8 f   MSVCRT:ucrt_stubs.obj
 0001:000031a8       __scrt_stub_for_acrt_thread_attach 00000001800041a8 f   MSVCRT:ucrt_stubs.obj
 0001:000031a8       __scrt_stub_for_acrt_thread_detach 00000001800041a8 f   MSVCRT:ucrt_stubs.obj
 0001:000031a8       __scrt_stub_for_acrt_uninitialize 00000001800041a8 f   MSVCRT:ucrt_stubs.obj
 0001:000031a8       __scrt_stub_for_acrt_uninitialize_critical 00000001800041a8 f   MSVCRT:ucrt_stubs.obj
 0001:000031a8       __vcrt_initialize          00000001800041a8 f   MSVCRT:ucrt_stubs.obj
 0001:000031a8       __vcrt_thread_attach       00000001800041a8 f   MSVCRT:ucrt_stubs.obj
 0001:000031a8       __vcrt_thread_detach       00000001800041a8 f   MSVCRT:ucrt_stubs.obj
 0001:000031a8       __vcrt_uninitialize        00000001800041a8 f   MSVCRT:ucrt_stubs.obj
 0001:000031a8       __vcrt_uninitialize_critical 00000001800041a8 f   MSVCRT:ucrt_stubs.obj
 0001:000031ac       __scrt_stub_for_is_c_termination_complete 00000001800041ac f   MSVCRT:ucrt_stubs.obj
 0001:000031ac       _is_c_termination_complete 00000001800041ac f   MSVCRT:ucrt_stubs.obj
 0001:000031c0       _guard_dispatch_icall_nop  00000001800041c0 f   MSVCRT:guard_dispatch.obj
 0001:000031e0       _guard_xfg_dispatch_icall_nop 00000001800041e0 f   MSVCRT:guard_xfg_dispatch.obj
 0002:00000000       __imp_RtlCaptureContext    0000000180005000     kernel32:KERNEL32.dll
 0002:00000008       __imp_RtlLookupFunctionEntry 0000000180005008     kernel32:KERNEL32.dll
 0002:00000010       __imp_RtlVirtualUnwind     0000000180005010     kernel32:KERNEL32.dll
 0002:00000018       __imp_UnhandledExceptionFilter 0000000180005018     kernel32:KERNEL32.dll
 0002:00000020       __imp_SetUnhandledExceptionFilter 0000000180005020     kernel32:KERNEL32.dll
 0002:00000028       __imp_GetCurrentProcess    0000000180005028     kernel32:KERNEL32.dll
 0002:00000030       __imp_TerminateProcess     0000000180005030     kernel32:KERNEL32.dll
 0002:00000038       __imp_IsProcessorFeaturePresent 0000000180005038     kernel32:KERNEL32.dll
 0002:00000040       __imp_CloseHandle          0000000180005040     kernel32:KERNEL32.dll
 0002:00000048       __imp_InitializeCriticalSectionAndSpinCount 0000000180005048     kernel32:KERNEL32.dll
 0002:00000050       __imp_DeleteCriticalSection 0000000180005050     kernel32:KERNEL32.dll
 0002:00000058       __imp_CreateEventW         0000000180005058     kernel32:KERNEL32.dll
 0002:00000060       __imp_GetModuleHandleW     0000000180005060     kernel32:KERNEL32.dll
 0002:00000068       __imp_GetProcAddress       0000000180005068     kernel32:KERNEL32.dll
 0002:00000070       __imp_IsDebuggerPresent    0000000180005070     kernel32:KERNEL32.dll
 0002:00000078       __imp_QueryPerformanceCounter 0000000180005078     kernel32:KERNEL32.dll
 0002:00000080       __imp_GetCurrentProcessId  0000000180005080     kernel32:KERNEL32.dll
 0002:00000088       __imp_GetCurrentThreadId   0000000180005088     kernel32:KERNEL32.dll
 0002:00000090       __imp_GetSystemTimeAsFileTime 0000000180005090     kernel32:KERNEL32.dll
 0002:00000098       __imp_DisableThreadLibraryCalls 0000000180005098     kernel32:KERNEL32.dll
 0002:000000a0       __imp_InitializeSListHead  00000001800050a0     kernel32:KERNEL32.dll
 0002:000000a8       \177KERNEL32_NULL_THUNK_DATA 00000001800050a8     kernel32:KERNEL32.dll
 0002:000000b0       __imp_memcpy               00000001800050b0     vcruntime:VCRUNTIME140.dll
 0002:000000b8       __imp_memset               00000001800050b8     vcruntime:VCRUNTIME140.dll
 0002:000000c0       __imp_strchr               00000001800050c0     vcruntime:VCRUNTIME140.dll
 0002:000000c8       __imp___C_specific_handler 00000001800050c8     vcruntime:VCRUNTIME140.dll
 0002:000000d0       __imp___std_type_info_destroy_list 00000001800050d0     vcruntime:VCRUNTIME140.dll
 0002:000000d8       \177VCRUNTIME140_NULL_THUNK_DATA 00000001800050d8     vcruntime:VCRUNTIME140.dll
 0002:000000e0       __imp_strtol               00000001800050e0     ucrt:api-ms-win-crt-convert-l1-1-0.dll
 0002:000000e8       \177api-ms-win-crt-convert-l1-1-0_NULL_THUNK_DATA 00000001800050e8     ucrt:api-ms-win-crt-convert-l1-1-0.dll
 0002:000000f0       __imp_malloc               00000001800050f0     ucrt:api-ms-win-crt-heap-l1-1-0.dll
 0002:000000f8       __imp_free                 00000001800050f8     ucrt:api-ms-win-crt-heap-l1-1-0.dll
 0002:00000100       \177api-ms-win-crt-heap-l1-1-0_NULL_THUNK_DATA 0000000180005100     ucrt:api-ms-win-crt-heap-l1-1-0.dll
 0002:00000108       __imp__errno               0000000180005108     ucrt:api-ms-win-crt-runtime-l1-1-0.dll
 0002:00000110       __imp_exit                 0000000180005110     ucrt:api-ms-win-crt-runtime-l1-1-0.dll
 0002:00000118       __imp__cexit               0000000180005118     ucrt:api-ms-win-crt-runtime-l1-1-0.dll
 0002:00000120       __imp__crt_atexit          0000000180005120     ucrt:api-ms-win-crt-runtime-l1-1-0.dll
 0002:00000128       __imp__execute_onexit_table 0000000180005128     ucrt:api-ms-win-crt-runtime-l1-1-0.dll
 0002:00000130       __imp__register_onexit_function 0000000180005130     ucrt:api-ms-win-crt-runtime-l1-1-0.dll
 0002:00000138       __imp__initialize_onexit_table 0000000180005138     ucrt:api-ms-win-crt-runtime-l1-1-0.dll
 0002:00000140       __imp__initialize_narrow_environment 0000000180005140     ucrt:api-ms-win-crt-runtime-l1-1-0.dll
 0002:00000148       __imp__configure_narrow_argv 0000000180005148     ucrt:api-ms-win-crt-runtime-l1-1-0.dll
 0002:00000150       __imp__seh_filter_dll      0000000180005150     ucrt:api-ms-win-crt-runtime-l1-1-0.dll
 0002:00000158       __imp__initterm_e          0000000180005158     ucrt:api-ms-win-crt-runtime-l1-1-0.dll
 0002:00000160       __imp__initterm            0000000180005160     ucrt:api-ms-win-crt-runtime-l1-1-0.dll
 0002:00000168       \177api-ms-win-crt-runtime-l1-1-0_NULL_THUNK_DATA 0000000180005168     ucrt:api-ms-win-crt-runtime-l1-1-0.dll
 0002:00000170       __imp___acrt_iob_func      0000000180005170     ucrt:api-ms-win-crt-stdio-l1-1-0.dll
 0002:00000178       __imp_fflush               0000000180005178     ucrt:api-ms-win-crt-stdio-l1-1-0.dll
 0002:00000180       __imp___stdio_common_vsprintf 0000000180005180     ucrt:api-ms-win-crt-stdio-l1-1-0.dll
 0002:00000188       __imp___stdio_common_vfprintf 0000000180005188     ucrt:api-ms-win-crt-stdio-l1-1-0.dll
 0002:00000190       \177api-ms-win-crt-stdio-l1-1-0_NULL_THUNK_DATA 0000000180005190     ucrt:api-ms-win-crt-stdio-l1-1-0.dll
 0002:00000198       __imp_strcmp               0000000180005198     ucrt:api-ms-win-crt-string-l1-1-0.dll
 0002:000001a0       __imp__strdup              00000001800051a0     ucrt:api-ms-win-crt-string-l1-1-0.dll
 0002:000001a0       __imp_strdup               00000001800051a0     ucrt:api-ms-win-crt-string-l1-1-0.dll
 0002:000001a8       __imp_strlen               00000001800051a8     ucrt:api-ms-win-crt-string-l1-1-0.dll
 0002:000001b0       __imp_strpbrk              00000001800051b0     ucrt:api-ms-win-crt-string-l1-1-0.dll
 0002:000001b8       __imp_strncpy              00000001800051b8     ucrt:api-ms-win-crt-string-l1-1-0.dll
 0002:000001c0       \177api-ms-win-crt-string-l1-1-0_NULL_THUNK_DATA 00000001800051c0     ucrt:api-ms-win-crt-string-l1-1-0.dll
 0002:000001c8       __guard_check_icall_fptr   00000001800051c8     MSVCRT:guard_support.obj
 0002:000001d0       __guard_xfg_check_icall_fptr 00000001800051d0     MSVCRT:guard_support.obj
 0002:000001d8       __guard_dispatch_icall_fptr 00000001800051d8     MSVCRT:guard_support.obj
 0002:000001e0       __guard_xfg_dispatch_icall_fptr 00000001800051e0     MSVCRT:guard_support.obj
 0002:000001e8       __guard_xfg_table_dispatch_icall_fptr 00000001800051e8     MSVCRT:guard_support.obj
 0002:000001f0       __castguard_check_failure_os_handled_fptr 00000001800051f0     MSVCRT:guard_support.obj
 0002:000001f8       __guard_memcpy_fptr        00000001800051f8     vcruntime:softmemtag.obj
 0002:00000200       __xc_a                     0000000180005200     MSVCRT:initializers.obj
 0002:00000208       __xc_z                     0000000180005208     MSVCRT:initializers.obj
 0002:00000210       __xi_a                     0000000180005210     MSVCRT:initializers.obj
 0002:00000220       __xi_z                     0000000180005220     MSVCRT:initializers.obj
 0002:00000228       __xl_a                     0000000180005228     MSVCRT:tlssup.obj
 0002:00000230       __xl_z                     0000000180005230     MSVCRT:tlssup.obj
 0002:00000238       __xp_a                     0000000180005238     MSVCRT:initializers.obj
 0002:00000240       __xp_z                     0000000180005240     MSVCRT:initializers.obj
 0002:00000248       __xt_a                     0000000180005248     MSVCRT:initializers.obj
 0002:00000250       __xt_z                     0000000180005250     MSVCRT:initializers.obj
 0002:00000260       g_refKindStr               0000000180005260     libSetNativeMethodPrefix002.obj
 0002:00000410       ??_C@_09BPLDFGCI@unknown_0@ 0000000180005410     libSetNativeMethodPrefix002.obj
 0002:00000420       ??_C@_0BL@FPNMECJD@JVMTI_HEAP_REFERENCE_CLASS@ 0000000180005420     libSetNativeMethodPrefix002.obj
 0002:00000440       ??_C@_0BL@FKGKKLNM@JVMTI_HEAP_REFERENCE_FIELD@ 0000000180005440     libSetNativeMethodPrefix002.obj
 0002:00000460       ??_C@_0CD@CAEHCFJF@JVMTI_HEAP_REFERENCE_ARRAY_ELEM@ 0000000180005460     libSetNativeMethodPrefix002.obj
 0002:00000488       ??_C@_0CC@DNEBMCNK@JVMTI_HEAP_REFERENCE_CLASS_LOAD@ 0000000180005488     libSetNativeMethodPrefix002.obj
 0002:000004b0       ??_C@_0BN@CJMIPEBB@JVMTI_HEAP_REFERENCE_SIGNERS@ 00000001800054b0     libSetNativeMethodPrefix002.obj
 0002:000004d0       ??_C@_0CH@HBOIDPEB@JVMTI_HEAP_REFERENCE_PROTECTION@ 00000001800054d0     libSetNativeMethodPrefix002.obj
 0002:000004f8       ??_C@_0BP@MDKGDGKL@JVMTI_HEAP_REFERENCE_INTERFACE@ 00000001800054f8     libSetNativeMethodPrefix002.obj
 0002:00000518       ??_C@_0CC@JJMIHNJH@JVMTI_HEAP_REFERENCE_STATIC_FIE@ 0000000180005518     libSetNativeMethodPrefix002.obj
 0002:00000540       ??_C@_0CD@IDHEEGID@JVMTI_HEAP_REFERENCE_CONSTANT_P@ 0000000180005540     libSetNativeMethodPrefix002.obj
 0002:00000568       ??_C@_0CA@EFFCHNG@JVMTI_HEAP_REFERENCE_SUPERCLASS@ 0000000180005568     libSetNativeMethodPrefix002.obj
 0002:00000588       ??_C@_0L@PCDFHGCJ@unknown_11@ 0000000180005588     libSetNativeMethodPrefix002.obj
 0002:00000598       ??_C@_0L@NJBICFOK@unknown_12@ 0000000180005598     libSetNativeMethodPrefix002.obj
 0002:000005a8       ??_C@_0L@MAADBEKL@unknown_13@ 00000001800055a8     libSetNativeMethodPrefix002.obj
 0002:000005b8       ??_C@_0L@IPECICGM@unknown_14@ 00000001800055b8     libSetNativeMethodPrefix002.obj
 0002:000005c8       ??_C@_0L@JGFJLDCN@unknown_15@ 00000001800055c8     libSetNativeMethodPrefix002.obj
 0002:000005d8       ??_C@_0L@LNHEOAOO@unknown_16@ 00000001800055d8     libSetNativeMethodPrefix002.obj
 0002:000005e8       ??_C@_0L@KEGPNBKP@unknown_17@ 00000001800055e8     libSetNativeMethodPrefix002.obj
 0002:000005f8       ??_C@_0L@CDPHMNGA@unknown_18@ 00000001800055f8     libSetNativeMethodPrefix002.obj
 0002:00000608       ??_C@_0L@DKOMPMCB@unknown_19@ 0000000180005608     libSetNativeMethodPrefix002.obj
 0002:00000618       ??_C@_0L@OJGIPJDB@unknown_20@ 0000000180005618     libSetNativeMethodPrefix002.obj
 0002:00000628       ??_C@_0CA@KAOFNDEM@JVMTI_HEAP_REFERENCE_JNI_GLOBAL@ 0000000180005628     libSetNativeMethodPrefix002.obj
 0002:00000648       ??_C@_0CC@HPFAJBK@JVMTI_HEAP_REFERENCE_SYSTEM_CLA@ 0000000180005648     libSetNativeMethodPrefix002.obj
 0002:00000670       ??_C@_0BN@FDEGFOHC@JVMTI_HEAP_REFERENCE_MONITOR@ 0000000180005670     libSetNativeMethodPrefix002.obj
 0002:00000690       ??_C@_0CB@HKIBCMAJ@JVMTI_HEAP_REFERENCE_STACK_LOCA@ 0000000180005690     libSetNativeMethodPrefix002.obj
 0002:000006b8       ??_C@_0BP@EAACMMOE@JVMTI_HEAP_REFERENCE_JNI_LOCAL@ 00000001800056b8     libSetNativeMethodPrefix002.obj
 0002:000006d8       ??_C@_0BM@IJDEOGOE@JVMTI_HEAP_REFERENCE_THREAD@ 00000001800056d8     libSetNativeMethodPrefix002.obj
 0002:000006f8       ??_C@_0BL@EDGPPKC@JVMTI_HEAP_REFERENCE_OTHER@ 00000001800056f8     libSetNativeMethodPrefix002.obj
 0002:00000714       ??_C@_04BCJPDBDA@Code@     0000000180005714     libSetNativeMethodPrefix002.obj
 0002:00000720       ??_C@_0BA@OCLMCFKC@LineNumberTable@ 0000000180005720     libSetNativeMethodPrefix002.obj
 0002:00000730       ??_C@_0BD@CPAEPILC@LocalVariableTable@ 0000000180005730     libSetNativeMethodPrefix002.obj
 0002:00000748       ??_C@_0BH@NMBDNHBD@LocalVariableTypeTable@ 0000000180005748     libSetNativeMethodPrefix002.obj
 0002:00000760       ??_C@_0O@HIHEEDNJ@StackMapTable@ 0000000180005760     libSetNativeMethodPrefix002.obj
 0002:00000770       ??_C@_0L@HCDIAMJG@?9?5?$CFs?0?5?$CFd?3?5@ 0000000180005770     libSetNativeMethodPrefix002.obj
 0002:00000780       ??_C@_0JI@HLPECLFI@?$CD?5?4?4?4?6?$CD?5ERROR?3?5too?5many?5complai@ 0000000180005780     libSetNativeMethodPrefix002.obj
 0002:00000820       ??_C@_0ED@JNEKCCOB@The?5following?5fake?5exception?5st@ 0000000180005820     libSetNativeMethodPrefix002.obj
 0002:00000868       ??_C@_0CN@FCNMDFBH@nsk?4share?4Fake_Exception_for_RU@ 0000000180005868     libSetNativeMethodPrefix002.obj
 0002:00000898       ??_C@_08PGFFNAEI@?$CI?$CFs?3?$CFd?$CJ?5@ 0000000180005898     libSetNativeMethodPrefix002.obj
 0002:000008a8       ??_C@_0DP@IENMAEGI@s?2test?2hotspot?2jtreg?2vmTestbase@ 00000001800058a8     libSetNativeMethodPrefix002.obj
 0002:000008e8       ??_C@_0BL@NDJLFFJB@?7at?5nsk_lvcomplain?$CI?$CFs?3?$CFd?$CJ?6@ 00000001800058e8     libSetNativeMethodPrefix002.obj
 0002:00000908       ??_C@_0BC@JOOKAFKF@?$CD?5ERROR?3?5?$CFs?0?5?$CFd?3?5@ 0000000180005908     libSetNativeMethodPrefix002.obj
 0002:00000920       ??_C@_09KJEAHMEH@?$CD?5ERROR?3?5@ 0000000180005920     libSetNativeMethodPrefix002.obj
 0002:0000092c       ??_C@_02GPIOPFAK@?$DO?$DO@ 000000018000592c     libSetNativeMethodPrefix002.obj
 0002:00000930       ??_C@_02FODMEDOG@?$DM?$DM@ 0000000180005930     libSetNativeMethodPrefix002.obj
 0002:00000934       ??_C@_02DJGKEECL@?4?4@     0000000180005934     libSetNativeMethodPrefix002.obj
 0002:00000938       ??_C@_0O@CJPGJOAF@?9?5?$CFs?0?5?$CFd?3?5?$CFs?5@ 0000000180005938     libSetNativeMethodPrefix002.obj
 0002:00000948       ??_C@_0CB@IAKPDOIC@?$CD?5?5?5verified?5assertion?5is?5FALSE@ 0000000180005948     libSetNativeMethodPrefix002.obj
 0002:00000970       ??_C@_0CO@LGONDEPD@stdout?3?5fflush?5failed?5?9?5err?$DN?$CFd?5@ 0000000180005970     libSetNativeMethodPrefix002.obj
 0002:000009a0       ??_C@_0CO@KBGKJPBD@stderr?3?5fflush?5failed?5?9?5err?$DN?$CFd?5@ 00000001800059a0     libSetNativeMethodPrefix002.obj
 0002:000009d0       ??_C@_0BB@JCNMKLLK@JVMTI_ERROR_NONE@ 00000001800059d0     libSetNativeMethodPrefix002.obj
 0002:000009e8       ??_C@_0BL@LDIMKLPH@JVMTI_ERROR_INVALID_THREAD@ 00000001800059e8     libSetNativeMethodPrefix002.obj
 0002:00000a08       ??_C@_0CB@PJFPAIKJ@JVMTI_ERROR_INVALID_THREAD_GROU@ 0000000180005a08     libSetNativeMethodPrefix002.obj
 0002:00000a30       ??_C@_0BN@LLMKHMNF@JVMTI_ERROR_INVALID_PRIORITY@ 0000000180005a30     libSetNativeMethodPrefix002.obj
 0002:00000a50       ??_C@_0CB@MBOFKAGB@JVMTI_ERROR_THREAD_NOT_SUSPENDE@ 0000000180005a50     libSetNativeMethodPrefix002.obj
 0002:00000a78       ??_C@_0BN@FABOLPBI@JVMTI_ERROR_THREAD_SUSPENDED@ 0000000180005a78     libSetNativeMethodPrefix002.obj
 0002:00000a98       ??_C@_0BN@FDGNOBJM@JVMTI_ERROR_THREAD_NOT_ALIVE@ 0000000180005a98     libSetNativeMethodPrefix002.obj
 0002:00000ab8       ??_C@_0BL@GOBIFKNJ@JVMTI_ERROR_INVALID_OBJECT@ 0000000180005ab8     libSetNativeMethodPrefix002.obj
 0002:00000ad8       ??_C@_0BK@FCMAJPPC@JVMTI_ERROR_INVALID_CLASS@ 0000000180005ad8     libSetNativeMethodPrefix002.obj
 0002:00000af8       ??_C@_0BP@IKLLBKEB@JVMTI_ERROR_CLASS_NOT_PREPARED@ 0000000180005af8     libSetNativeMethodPrefix002.obj
 0002:00000b18       ??_C@_0BN@KLPPLKG@JVMTI_ERROR_INVALID_METHODID@ 0000000180005b18     libSetNativeMethodPrefix002.obj
 0002:00000b38       ??_C@_0BN@BCEKOKND@JVMTI_ERROR_INVALID_LOCATION@ 0000000180005b38     libSetNativeMethodPrefix002.obj
 0002:00000b58       ??_C@_0BM@DFDGPME@JVMTI_ERROR_INVALID_FIELDID@ 0000000180005b58     libSetNativeMethodPrefix002.obj
 0002:00000b78       ??_C@_0BL@NELIEPEC@JVMTI_ERROR_NO_MORE_FRAMES@ 0000000180005b78     libSetNativeMethodPrefix002.obj
 0002:00000b98       ??_C@_0BJ@BDBECFDM@JVMTI_ERROR_OPAQUE_FRAME@ 0000000180005b98     libSetNativeMethodPrefix002.obj
 0002:00000bb8       ??_C@_0BK@MIIFNLOB@JVMTI_ERROR_TYPE_MISMATCH@ 0000000180005bb8     libSetNativeMethodPrefix002.obj
 0002:00000bd8       ??_C@_0BJ@HPCAOILC@JVMTI_ERROR_INVALID_SLOT@ 0000000180005bd8     libSetNativeMethodPrefix002.obj
 0002:00000bf8       ??_C@_0BG@CHILOPNI@JVMTI_ERROR_DUPLICATE@ 0000000180005bf8     libSetNativeMethodPrefix002.obj
 0002:00000c10       ??_C@_0BG@DIEMLHKM@JVMTI_ERROR_NOT_FOUND@ 0000000180005c10     libSetNativeMethodPrefix002.obj
 0002:00000c28       ??_C@_0BM@NHMCKHOB@JVMTI_ERROR_INVALID_MONITOR@ 0000000180005c28     libSetNativeMethodPrefix002.obj
 0002:00000c48       ??_C@_0BO@PPEDAJGL@JVMTI_ERROR_NOT_MONITOR_OWNER@ 0000000180005c48     libSetNativeMethodPrefix002.obj
 0002:00000c68       ??_C@_0BG@FCAIPEID@JVMTI_ERROR_INTERRUPT@ 0000000180005c68     libSetNativeMethodPrefix002.obj
 0002:00000c80       ??_C@_0CB@EGDBNKOI@JVMTI_ERROR_INVALID_CLASS_FORMA@ 0000000180005c80     libSetNativeMethodPrefix002.obj
 0002:00000ca8       ??_C@_0CG@DGKOGIAL@JVMTI_ERROR_CIRCULAR_CLASS_DEFI@ 0000000180005ca8     libSetNativeMethodPrefix002.obj
 0002:00000cd0       ??_C@_0BP@ICEALPKC@JVMTI_ERROR_FAILS_VERIFICATION@ 0000000180005cd0     libSetNativeMethodPrefix002.obj
 0002:00000cf0       ??_C@_0DC@JDACLMIO@JVMTI_ERROR_UNSUPPORTED_REDEFIN@ 0000000180005cf0     libSetNativeMethodPrefix002.obj
 0002:00000d28       ??_C@_0DE@GKDKNOMJ@JVMTI_ERROR_UNSUPPORTED_REDEFIN@ 0000000180005d28     libSetNativeMethodPrefix002.obj
 0002:00000d60       ??_C@_0BO@LAFKIOG@JVMTI_ERROR_INVALID_TYPESTATE@ 0000000180005d60     libSetNativeMethodPrefix002.obj
 0002:00000d80       ??_C@_0DH@INDGCLLB@JVMTI_ERROR_UNSUPPORTED_REDEFIN@ 0000000180005d80     libSetNativeMethodPrefix002.obj
 0002:00000db8       ??_C@_0DE@NHEOMMGI@JVMTI_ERROR_UNSUPPORTED_REDEFIN@ 0000000180005db8     libSetNativeMethodPrefix002.obj
 0002:00000df0       ??_C@_0CA@EKPNJOEP@JVMTI_ERROR_UNSUPPORTED_VERSION@ 0000000180005df0     libSetNativeMethodPrefix002.obj
 0002:00000e10       ??_C@_0BN@OFFMAHHL@JVMTI_ERROR_NAMES_DONT_MATCH@ 0000000180005e10     libSetNativeMethodPrefix002.obj
 0002:00000e30       ??_C@_0DN@HHBBLAKE@JVMTI_ERROR_UNSUPPORTED_REDEFIN@ 0000000180005e30     libSetNativeMethodPrefix002.obj
 0002:00000e70       ??_C@_0DO@HMBGBGNA@JVMTI_ERROR_UNSUPPORTED_REDEFIN@ 0000000180005e70     libSetNativeMethodPrefix002.obj
 0002:00000eb0       ??_C@_0BP@PBECGKHJ@JVMTI_ERROR_UNMODIFIABLE_CLASS@ 0000000180005eb0     libSetNativeMethodPrefix002.obj
 0002:00000ed0       ??_C@_0BK@CANILEHF@JVMTI_ERROR_NOT_AVAILABLE@ 0000000180005ed0     libSetNativeMethodPrefix002.obj
 0002:00000ef0       ??_C@_0CE@INJKMEFK@JVMTI_ERROR_MUST_POSSESS_CAPABI@ 0000000180005ef0     libSetNativeMethodPrefix002.obj
 0002:00000f18       ??_C@_0BJ@LBFPFPDM@JVMTI_ERROR_NULL_POINTER@ 0000000180005f18     libSetNativeMethodPrefix002.obj
 0002:00000f38       ??_C@_0BP@CHJPNNEM@JVMTI_ERROR_ABSENT_INFORMATION@ 0000000180005f38     libSetNativeMethodPrefix002.obj
 0002:00000f58       ??_C@_0BP@OMFMNLC@JVMTI_ERROR_INVALID_EVENT_TYPE@ 0000000180005f58     libSetNativeMethodPrefix002.obj
 0002:00000f78       ??_C@_0BN@BIBNPHHO@JVMTI_ERROR_ILLEGAL_ARGUMENT@ 0000000180005f78     libSetNativeMethodPrefix002.obj
 0002:00000f98       ??_C@_0BK@KKNDHDCE@JVMTI_ERROR_NATIVE_METHOD@ 0000000180005f98     libSetNativeMethodPrefix002.obj
 0002:00000fb8       ??_C@_0BK@PMKCFHAE@JVMTI_ERROR_OUT_OF_MEMORY@ 0000000180005fb8     libSetNativeMethodPrefix002.obj
 0002:00000fd8       ??_C@_0BK@NNJBDMNB@JVMTI_ERROR_ACCESS_DENIED@ 0000000180005fd8     libSetNativeMethodPrefix002.obj
 0002:00000ff8       ??_C@_0BI@GHECLMNC@JVMTI_ERROR_WRONG_PHASE@ 0000000180005ff8     libSetNativeMethodPrefix002.obj
 0002:00001010       ??_C@_0BF@OLIHJOII@JVMTI_ERROR_INTERNAL@ 0000000180006010     libSetNativeMethodPrefix002.obj
 0002:00001028       ??_C@_0BO@EOHGKJHI@JVMTI_ERROR_UNATTACHED_THREAD@ 0000000180006028     libSetNativeMethodPrefix002.obj
 0002:00001048       ??_C@_0CA@LKHFDACL@JVMTI_ERROR_INVALID_ENVIRONMENT@ 0000000180006048     libSetNativeMethodPrefix002.obj
 0002:00001068       ??_C@_0BA@MMFHLOKK@?$DMunknown?5error?$DO@ 0000000180006068     libSetNativeMethodPrefix002.obj
 0002:00001078       ??_C@_0CF@CBHOKDB@throwable?5?$DN?5jni?9?$DOExceptionOccur@ 0000000180006078     libSetNativeMethodPrefix002.obj
 0002:000010a0       ??_C@_03OFAPEBGM@?$CFs?6@  00000001800060a0     libSetNativeMethodPrefix002.obj
 0002:000010a8       ??_C@_0DM@LPIGEGNJ@s?2test?2hotspot?2jtreg?2vmTestbase@ 00000001800060a8     libSetNativeMethodPrefix002.obj
 0002:000010e8       ??_C@_0CC@NFCNPEPK@Exception?5in?5JNI?5call?5?$CIcleared?$CJ@ 00000001800060e8     libSetNativeMethodPrefix002.obj
 0002:00001110       ??_C@_0BJ@IBAKFIKF@jni?9?$DOExceptionDescribe?$CI?$CJ@ 0000000180006110     libSetNativeMethodPrefix002.obj
 0002:00001130       ??_C@_0BG@GGKALKMH@jni?9?$DOExceptionClear?$CI?$CJ@ 0000000180006130     libSetNativeMethodPrefix002.obj
 0002:00001148       ??_C@_0CF@JMGFGJLJ@?$CD?5?5?5verified?5JNI?5assertion?5is?5F@ 0000000180006148     libSetNativeMethodPrefix002.obj
 0002:00001170       ??_C@_07KBAMPNJK@verbose@  0000000180006170     libSetNativeMethodPrefix002.obj
 0002:00001178       ??_C@_0DN@PKJBOLAP@nsk_jvmti_parseOptions?$CI?$CJ?3?5unexp@ 0000000180006178     libSetNativeMethodPrefix002.obj
 0002:000011b8       ??_C@_05IMBNNINJ@trace@    00000001800061b8     libSetNativeMethodPrefix002.obj
 0002:000011c0       ??_C@_0DD@BJKGNDMB@nsk_jvmti_parseOptions?$CI?$CJ?3?5no?5va@ 00000001800061c0     libSetNativeMethodPrefix002.obj
 0002:000011f4       ??_C@_04CGFJFPFD@none@     00000001800061f4     libSetNativeMethodPrefix002.obj
 0002:000011fc       ??_C@_06BMELKFMA@before@   00000001800061fc     libSetNativeMethodPrefix002.obj
 0002:00001204       ??_C@_05CMKPCFDK@after@    0000000180006204     libSetNativeMethodPrefix002.obj
 0002:0000120c       ??_C@_03NFKEKGGK@all@      000000018000620c     libSetNativeMethodPrefix002.obj
 0002:00001210       ??_C@_0DM@NDNJGJKE@nsk_jvmti_parseOptions?$CI?$CJ?3?5uexpe@ 0000000180006210     libSetNativeMethodPrefix002.obj
 0002:00001250       ??_C@_08NBBJKJO@waittime@  0000000180006250     libSetNativeMethodPrefix002.obj
 0002:00001260       ??_C@_0DO@CMHGAOHC@nsk_jvmti_parseOptions?$CI?$CJ?3?5not?5i@ 0000000180006260     libSetNativeMethodPrefix002.obj
 0002:000012a0       ??_C@_0DL@LNMPBDLN@nsk_jvmti_parseOptions?$CI?$CJ?3?5negat@ 00000001800062a0     libSetNativeMethodPrefix002.obj
 0002:000012e0       ??_C@_0DA@GMFJNOJH@nsk_jvmti_parseOptions?$CI?$CJ?3?5unkno@ 00000001800062e0     libSetNativeMethodPrefix002.obj
 0002:00001310       ??_C@_0CO@CCIAMEAN@nsk_jvmti_parseOptions?$CI?$CJ?3?5found@ 0000000180006310     libSetNativeMethodPrefix002.obj
 0002:00001340       ??_C@_0CJ@OEGPCGDL@nsk_jvmti_parseOptions?$CI?$CJ?3?5out?5o@ 0000000180006340     libSetNativeMethodPrefix002.obj
 0002:00001370       ??_C@_0DI@NMBHPGGF@nsk_jvmti_parseOptions?$CI?$CJ?3?5too?5m@ 0000000180006370     libSetNativeMethodPrefix002.obj
 0002:000013a8       ??_C@_03POGCGECB@?5?0?$HO@ 00000001800063a8     libSetNativeMethodPrefix002.obj
 0002:000013b0       ??_C@_0DC@GKLNPJIJ@nsk_jvmti_findOptionValue?$CI?$CJ?3?5op@ 00000001800063b0     libSetNativeMethodPrefix002.obj
 0002:000013e8       ??_C@_0DF@OPPIHBPJ@nsk_jvmti_findOptionIntValue?$CI?$CJ?3@ 00000001800063e8     libSetNativeMethodPrefix002.obj
 0002:00001420       ??_C@_0DO@DBKDODPI@nsk_jvmti_findOptionIntValue?$CI?$CJ?3@ 0000000180006420     libSetNativeMethodPrefix002.obj
 0002:00001460       ??_C@_0EE@NGNPKOJC@nsk_jvmti_findOptionIntValue?$CI?$CJ?3@ 0000000180006460     libSetNativeMethodPrefix002.obj
 0002:000014a8       ??_C@_0CB@MLNJNCLJ@?5?5jvmti?5error?3?5code?$DN?$CFd?0?5name?$DN?$CFs@ 00000001800064a8     libSetNativeMethodPrefix002.obj
 0002:000014d0       ??_C@_0CD@OHBGDKMK@?$CD?5?5?5jvmti?5error?3?5code?$DN?$CFd?0?5name?$DN@ 00000001800064d0     libSetNativeMethodPrefix002.obj
 0002:000014f8       ??_C@_0CG@JNNCGPHB@?$CD?5?5?5error?5expected?3?5code?$DN?$CFd?0?5na@ 00000001800064f8     libSetNativeMethodPrefix002.obj
 0002:00001520       ??_C@_0EB@IMGKPCGE@?$CIstr_obj?5?$DN?5jni?9?$DONewStringUTF?$CIco@ 0000000180006520     libSetNativeMethodPrefix002.obj
 0002:00001570       ??_C@_0EA@HFOGGBCC@s?2test?2hotspot?2jtreg?2vmTestbase@ 0000000180006570     libSetNativeMethodPrefix002.obj
 0002:000015b0       ??_C@_05KKCIMGE@error@     00000001800065b0     libSetNativeMethodPrefix002.obj
 0002:000015b8       ??_C@_0BD@HGNAOMCP@agent_data_monitor@ 00000001800065b8     libSetNativeMethodPrefix002.obj
 0002:000015d0       ??_C@_0EB@OGCLGKLN@javaVM?9?$DOGetEnv?$CI?$CIvoid?5?$CK?$CK?$CJ?$CGjvmti_@ 00000001800065d0     libSetNativeMethodPrefix002.obj
 0002:00001620       ??_C@_0EA@PNBCDMOA@s?2test?2hotspot?2jtreg?2vmTestbase@ 0000000180006620     libSetNativeMethodPrefix002.obj
 0002:00001660       ??_C@_0CI@DDPIFBGM@init_agent_data?$CIjvmti_env?0?5?$CGage@ 0000000180006660     libSetNativeMethodPrefix002.obj
 0002:00001688       ??_C@_0DI@ILAHDLMP@?$CI?$CKagentThreadProc?$CJ?$CIjvmti_env?0?5a@ 0000000180006688     libSetNativeMethodPrefix002.obj
 0002:000016c0       ??_C@_0BD@KDBALNLB@JVMTI?5agent?5thread@ 00000001800066c0     libSetNativeMethodPrefix002.obj
 0002:000016d8       ??_C@_0BB@NOKBFPFO@java?1lang?1Thread@ 00000001800066d8     libSetNativeMethodPrefix002.obj
 0002:000016ec       ??_C@_06FALKBLGB@?$DMinit?$DO@ 00000001800066ec     libSetNativeMethodPrefix002.obj
 0002:000016f8       ??_C@_0BG@IKDDPPGD@?$CILjava?1lang?1String?$DL?$CJV@ 00000001800066f8     libSetNativeMethodPrefix002.obj
 0002:00001710       ??_C@_0EB@IFJBFEKC@?$CIthreadClass?5?$DN?5jni_env?9?$DOFindCla@ 0000000180006710     libSetNativeMethodPrefix002.obj
 0002:00001760       ??_C@_0GF@FGFIBKKL@?$CIthreadCtor?5?$DN?5jni_env?9?$DOGetMetho@ 0000000180006760     libSetNativeMethodPrefix002.obj
 0002:000017c8       ??_C@_0DN@NCPDJLOG@?$CIthreadName?5?$DN?5jni_env?9?$DONewStrin@ 00000001800067c8     libSetNativeMethodPrefix002.obj
 0002:00001810       ??_C@_0FE@PFKODBGC@?$CIthreadObject?5?$DN?5jni_env?9?$DONewObj@ 0000000180006810     libSetNativeMethodPrefix002.obj
 0002:00001870       ??_C@_0ED@HOBAHHJI@?$CIthreadGlobalRef?5?$DN?5jni_env?9?$DONew@ 0000000180006870     libSetNativeMethodPrefix002.obj
 0002:000018c0       ??_C@_0FN@HNJJAHFC@jvmti_env?9?$DORunAgentThread?$CIagent@ 00000001800068c0     libSetNativeMethodPrefix002.obj
 0002:00001920       ??_C@_0EA@MOJDNKDF@Debuggee?5status?5sync?5aborted?5be@ 0000000180006920     libSetNativeMethodPrefix002.obj
 0002:00001960       ??_C@_0EA@EEOEJAEN@status?5?$DN?5syncDebuggeeStatus?$CIjni@ 0000000180006960     libSetNativeMethodPrefix002.obj
 0002:000019a0       ??_C@_0BL@JBCFNBMB@nsk_jvmti_resetAgentData?$CI?$CJ@ 00000001800069a0     libSetNativeMethodPrefix002.obj
 0002:000019c0       ??_C@_0EL@LPBEELIP@s?2test?2hotspot?2jtreg?2vmTestbase@ 00000001800069c0     libSetNativeMethodPrefix002.obj
 0002:00001a10       ??_C@_0CK@JDAMFDMJ@jvmti?9?$DOSetTag?$CIo?0?5tag?$CJ?5?$DN?$DN?5JVMTI_@ 0000000180006a10     libSetNativeMethodPrefix002.obj
 0002:00001a40       ??_C@_0CC@DAMNHKNI@Can?8t?5set?5tag?5?$CFli?5for?5object?5?$CFl@ 0000000180006a40     libSetNativeMethodPrefix002.obj
 0002:00001a68       ??_C@_0DL@HAJPNKEF@jvmti?9?$DOGetObjectHashCode?$CIo?0?5?$CGha@ 0000000180006a68     libSetNativeMethodPrefix002.obj
 0002:00001aa8       ??_C@_0BL@JFPIEOBF@Can?8t?5get?5hash?5object?5?$CFlx?6@ 0000000180006aa8     libSetNativeMethodPrefix002.obj
 0002:00001ac8       ??_C@_0BG@DICPHBKN@setTag?3?5?$CF08x?5?$DM?9?5?$CF?53li@ 0000000180006ac8     libSetNativeMethodPrefix002.obj
 0002:00001ae0       ??_C@_0DH@FCEEBDMJ@?$CIs?5?$DN?5jni?9?$DOGetStringUTFChars?$CIsIn@ 0000000180006ae0     libSetNativeMethodPrefix002.obj
 0002:00001b18       ??_C@_0BJ@OKKGHDCN@Can?8t?5get?5string?5at?5?$CF?$CDp?6@ 0000000180006b18     libSetNativeMethodPrefix002.obj
 0002:00001b38       ??_C@_0BP@EKFLGGFJ@Can?8t?5get?5string?5at?5?$CF?$CDp?3?5null?6@ 0000000180006b38     libSetNativeMethodPrefix002.obj
 0002:00001b58       ??_C@_06ICODBHCL@?5?1?1?5?$CFs@ 0000000180006b58     libSetNativeMethodPrefix002.obj
 0002:00001b60       ??_C@_0DB@KGFPLEGO@?$CIr?5?$DN?5jvmti?9?$DOGetTag?$CIo?0?5?$CGtag?$CJ?$CJ?5?$DN?$DN@ 0000000180006b60     libSetNativeMethodPrefix002.obj
 0002:00001b98       ??_C@_0CO@PDAGBCGJ@Can?8t?5GetTag?5for?5object?5?$CFlx?4?5Re@ 0000000180006b98     libSetNativeMethodPrefix002.obj
 0002:00001bc8       ??_C@_0CH@HPEODOHC@TEST_BUG?3?5Max?4?5number?5of?5refs?5r@ 0000000180006bc8     libSetNativeMethodPrefix002.obj
 0002:00001bf0       ??_C@_0DI@PHFCABIM@?$CIr?5?$DN?5jvmti?9?$DOGetTag?$CIfrom?0?5?$CGtagFr@ 0000000180006bf0     libSetNativeMethodPrefix002.obj
 0002:00001c28       ??_C@_0DI@MDEGFNKD@TEST_BUG?3?5Can?8t?5GetTag?5for?5obje@ 0000000180006c28     libSetNativeMethodPrefix002.obj
 0002:00001c60       ??_C@_0DE@MLELJAHM@?$CIr?5?$DN?5jvmti?9?$DOGetTag?$CIto?0?5?$CGtagTo?$CJ?$CJ@ 0000000180006c60     libSetNativeMethodPrefix002.obj
 0002:00001ca0       ??_C@_0EK@PDFHNKHB@?5?$DO?$DO?$DO?5SetNativeMethodPrefix002?4f@ 0000000180006ca0     libSetNativeMethodPrefix002.obj
 0002:00001cf0       ??_C@_0HG@DBAMOJPE@s?2test?2hotspot?2jtreg?2vmTestbase@ 0000000180006cf0     libSetNativeMethodPrefix002.obj
 0002:00001d68       ??_C@_0CF@JPCDCNOC@jvmti?9?$DOSetNativeMethodPrefix?$CIpr@ 0000000180006d68     libSetNativeMethodPrefix002.obj
 0002:00001d90       ??_C@_0CA@MNKGCBCG@nsk_jvmti_parseOptions?$CIoptions?$CJ@ 0000000180006d90     libSetNativeMethodPrefix002.obj
 0002:00001db0       ??_C@_06CHGOAPND@prefix@   0000000180006db0     libSetNativeMethodPrefix002.obj
 0002:00001db8       ??_C@_0M@EJBPPACI@Prefix?3?5?$CFs?6@ 0000000180006db8     libSetNativeMethodPrefix002.obj
 0002:00001dc4       ??_C@_05KAEIDCAL@apply@    0000000180006dc4     libSetNativeMethodPrefix002.obj
 0002:00001dd0       ??_C@_0DM@OFHPOAIH@?$CIjvmti?5?$DN?5nsk_jvmti_createJVMTIE@ 0000000180006dd0     libSetNativeMethodPrefix002.obj
 0002:00001e10       ??_C@_0BO@IAKFILDF@jvmti?9?$DOGetCapabilities?$CI?$CGcaps?$CJ@ 0000000180006e10     libSetNativeMethodPrefix002.obj
 0002:00001e30       ??_C@_0BO@DBKDIPGD@jvmti?9?$DOAddCapabilities?$CI?$CGcaps?$CJ@ 0000000180006e30     libSetNativeMethodPrefix002.obj
 0002:00001e50       ??_C@_0CP@FKCHNNAC@Can?8t?5specify?5prefix?5for?5native@ 0000000180006e50     libSetNativeMethodPrefix002.obj
 0002:00001e90       ??_C@_1EC@JIJBPKFM@?$AAa?$AAp?$AAi?$AA?9?$AAm?$AAs?$AA?9?$AAw?$AAi?$AAn?$AA?9?$AAc?$AAo?$AAr?$AAe@ 0000000180006e90     MSVCRT:thread_safe_statics.obj
 0002:00001ed8       ??_C@_1BK@MGMFAEKH@?$AAk?$AAe?$AAr?$AAn?$AAe?$AAl?$AA3?$AA2?$AA?4?$AAd?$AAl?$AAl@ 0000000180006ed8     MSVCRT:thread_safe_statics.obj
 0002:00001ef8       ??_C@_0BJ@JEBJOJFJ@SleepConditionVariableCS@ 0000000180006ef8     MSVCRT:thread_safe_statics.obj
 0002:00001f18       ??_C@_0BJ@PGPPEPCC@WakeAllConditionVariable@ 0000000180006f18     MSVCRT:thread_safe_statics.obj
 0002:00001f38       _pDefaultRawDllMain        0000000180006f38     MSVCRT:dll_dllmain.obj
 0002:00001f38       _pRawDllMain               0000000180006f38     MSVCRT:dll_dllmain.obj
 0002:00001f40       __xmm@ffffffffffffffffffffffffffffffff 0000000180006f40     MSVCRT:utility.obj
 0002:00001f50       _load_config_used          0000000180006f50     MSVCRT:loadcfg.obj
 0002:00002100       _tls_used                  0000000180007100     MSVCRT:tlssup.obj
 0002:00002128       __volatile_metadata        0000000180007128     <linker-defined>
 0002:00002508       __rtc_iaa                  0000000180007508     MSVCRT:initsect.obj
 0002:00002510       __rtc_izz                  0000000180007510     MSVCRT:initsect.obj
 0002:00002518       __rtc_taa                  0000000180007518     MSVCRT:initsect.obj
 0002:00002520       __rtc_tzz                  0000000180007520     MSVCRT:initsect.obj
 0002:00002528       _tls_start                 0000000180007528     MSVCRT:tlssup.obj
 0002:0000252c       _Init_thread_epoch         000000018000752c     MSVCRT:thread_safe_statics.obj
 0002:00002530       _tls_end                   0000000180007530     MSVCRT:tlssup.obj
 0002:00002c2c       __IMPORT_DESCRIPTOR_KERNEL32 0000000180007c2c     kernel32:KERNEL32.dll
 0002:00002c40       __IMPORT_DESCRIPTOR_VCRUNTIME140 0000000180007c40     vcruntime:VCRUNTIME140.dll
 0002:00002c54       __IMPORT_DESCRIPTOR_api-ms-win-crt-heap-l1-1-0 0000000180007c54     ucrt:api-ms-win-crt-heap-l1-1-0.dll
 0002:00002c68       __IMPORT_DESCRIPTOR_api-ms-win-crt-runtime-l1-1-0 0000000180007c68     ucrt:api-ms-win-crt-runtime-l1-1-0.dll
 0002:00002c7c       __IMPORT_DESCRIPTOR_api-ms-win-crt-convert-l1-1-0 0000000180007c7c     ucrt:api-ms-win-crt-convert-l1-1-0.dll
 0002:00002c90       __IMPORT_DESCRIPTOR_api-ms-win-crt-stdio-l1-1-0 0000000180007c90     ucrt:api-ms-win-crt-stdio-l1-1-0.dll
 0002:00002ca4       __IMPORT_DESCRIPTOR_api-ms-win-crt-string-l1-1-0 0000000180007ca4     ucrt:api-ms-win-crt-string-l1-1-0.dll
 0002:00002cb8       __NULL_IMPORT_DESCRIPTOR   0000000180007cb8     kernel32:KERNEL32.dll
 0003:00000030       _Init_global_epoch         0000000180009030     MSVCRT:thread_safe_statics.obj
 0003:00000040       __security_cookie          0000000180009040     MSVCRT:gs_cookie.obj
 0003:00000048       __security_cookie_complement 0000000180009048     MSVCRT:gs_cookie.obj
 0003:00000050       __scrt_native_dllmain_reason 0000000180009050     MSVCRT:utility.obj
 0003:00000058       __isa_available            0000000180009058     MSVCRT:cpu_disp.obj
 0003:0000005c       __isa_enabled              000000018000905c     MSVCRT:cpu_disp.obj
 0003:00000060       __memset_fast_string_threshold 0000000180009060     MSVCRT:cpu_disp.obj
 0003:00000068       __memset_nt_threshold      0000000180009068     MSVCRT:cpu_disp.obj
 0003:00000070       __scrt_ucrt_dll_is_in_use  0000000180009070     MSVCRT:ucrt_stubs.obj
 0003:00000080       g_wrongHeapCallbacks       0000000180009080     libSetNativeMethodPrefix002.obj
 0003:00000100       g_szTagInfo                0000000180009100     libSetNativeMethodPrefix002.obj
 0003:00002040       g_tagFlags                 000000018000b040     libSetNativeMethodPrefix002.obj
 0003:00002428       g_refsToVerifyCnt          000000018000b428     libSetNativeMethodPrefix002.obj
 0003:0000242c       g_fakeUserData             000000018000b42c     libSetNativeMethodPrefix002.obj
 0003:00002430       g_tagVisitCount            000000018000b430     libSetNativeMethodPrefix002.obj
 0003:000033d0       g_refsToVerify             000000018000c3d0     libSetNativeMethodPrefix002.obj
 0003:0001aad0       g_userDataError            0000000180023ad0     libSetNativeMethodPrefix002.obj
 0003:0001ac78       ?_OptionsStorage@?1??__local_stdio_printf_options@@9@4_KA 0000000180023c78     libSetNativeMethodPrefix002.obj
 0003:0001b238       _tls_index                 0000000180024238     MSVCRT:tlssup.obj
 0003:0001b240       __scrt_current_native_startup_state 0000000180024240     MSVCRT:utility.obj
 0003:0001b248       __scrt_native_startup_lock 0000000180024248     MSVCRT:utility.obj
 0003:0001b288       __scrt_debugger_hook_flag  0000000180024288     MSVCRT:utility_desktop.obj
 0003:0001b290       ?__type_info_root_node@@3U__type_info_node@@A 0000000180024290     MSVCRT:tncleanup.obj
 0003:0001b2a0       ?_OptionsStorage@?1??__local_stdio_scanf_options@@9@4_KA 00000001800242a0     MSVCRT:default_local_stdio_options.obj
 0003:0001b2a8       __favor                    00000001800242a8     MSVCRT:cpu_disp.obj
 0003:0001b2b0       __dyn_tls_init_callback    00000001800242b0     <common>

 entry point at        0001:000028d0

 Static symbols

 0000:fffd9000       .debug$S                   0000000180000000     SetNativeMethodPrefix002.exp
 0000:fffd9000       .debug$S                   0000000180000000     vcruntime:VCRUNTIME140.dll
 0000:fffd9000       .debug$S                   0000000180000000     vcruntime:VCRUNTIME140.dll
 0000:fffd9000       .debug$S                   0000000180000000     vcruntime:VCRUNTIME140.dll
 0000:fffd9000       .debug$S                   0000000180000000     vcruntime:VCRUNTIME140.dll
 0000:fffd9000       .debug$S                   0000000180000000     vcruntime:VCRUNTIME140.dll
 0000:fffd9000       .debug$S                   0000000180000000     vcruntime:VCRUNTIME140.dll
 0000:fffd9000       .debug$S                   0000000180000000     vcruntime:VCRUNTIME140.dll
 0000:fffd9000       .debug$S                   0000000180000000     ucrt:api-ms-win-crt-convert-l1-1-0.dll
 0000:fffd9000       .debug$S                   0000000180000000     ucrt:api-ms-win-crt-heap-l1-1-0.dll
 0000:fffd9000       .debug$S                   0000000180000000     ucrt:api-ms-win-crt-heap-l1-1-0.dll
 0000:fffd9000       .debug$S                   0000000180000000     ucrt:api-ms-win-crt-heap-l1-1-0.dll
 0000:fffd9000       .debug$S                   0000000180000000     ucrt:api-ms-win-crt-heap-l1-1-0.dll
 0000:fffd9000       .debug$S                   0000000180000000     ucrt:api-ms-win-crt-runtime-l1-1-0.dll
 0000:fffd9000       .debug$S                   0000000180000000     ucrt:api-ms-win-crt-runtime-l1-1-0.dll
 0000:fffd9000       .debug$S                   0000000180000000     ucrt:api-ms-win-crt-runtime-l1-1-0.dll
 0000:fffd9000       .debug$S                   0000000180000000     ucrt:api-ms-win-crt-runtime-l1-1-0.dll
 0000:fffd9000       .debug$S                   0000000180000000     ucrt:api-ms-win-crt-runtime-l1-1-0.dll
 0000:fffd9000       .debug$S                   0000000180000000     ucrt:api-ms-win-crt-runtime-l1-1-0.dll
 0000:fffd9000       .debug$S                   0000000180000000     ucrt:api-ms-win-crt-runtime-l1-1-0.dll
 0000:fffd9000       .debug$S                   0000000180000000     ucrt:api-ms-win-crt-runtime-l1-1-0.dll
 0000:fffd9000       .debug$S                   0000000180000000     ucrt:api-ms-win-crt-runtime-l1-1-0.dll
 0000:fffd9000       .debug$S                   0000000180000000     ucrt:api-ms-win-crt-runtime-l1-1-0.dll
 0000:fffd9000       .debug$S                   0000000180000000     ucrt:api-ms-win-crt-runtime-l1-1-0.dll
 0000:fffd9000       .debug$S                   0000000180000000     ucrt:api-ms-win-crt-runtime-l1-1-0.dll
 0000:fffd9000       .debug$S                   0000000180000000     ucrt:api-ms-win-crt-runtime-l1-1-0.dll
 0000:fffd9000       .debug$S                   0000000180000000     ucrt:api-ms-win-crt-runtime-l1-1-0.dll
 0000:fffd9000       .debug$S                   0000000180000000     ucrt:api-ms-win-crt-runtime-l1-1-0.dll
 0000:fffd9000       .debug$S                   0000000180000000     ucrt:api-ms-win-crt-runtime-l1-1-0.dll
 0000:fffd9000       .debug$S                   0000000180000000     ucrt:api-ms-win-crt-stdio-l1-1-0.dll
 0000:fffd9000       .debug$S                   0000000180000000     ucrt:api-ms-win-crt-stdio-l1-1-0.dll
 0000:fffd9000       .debug$S                   0000000180000000     ucrt:api-ms-win-crt-stdio-l1-1-0.dll
 0000:fffd9000       .debug$S                   0000000180000000     ucrt:api-ms-win-crt-stdio-l1-1-0.dll
 0000:fffd9000       .debug$S                   0000000180000000     ucrt:api-ms-win-crt-stdio-l1-1-0.dll
 0000:fffd9000       .debug$S                   0000000180000000     ucrt:api-ms-win-crt-stdio-l1-1-0.dll
 0000:fffd9000       .debug$S                   0000000180000000     ucrt:api-ms-win-crt-stdio-l1-1-0.dll
 0000:fffd9000       .debug$S                   0000000180000000     ucrt:api-ms-win-crt-stdio-l1-1-0.dll
 0000:fffd9000       .debug$S                   0000000180000000     ucrt:api-ms-win-crt-stdio-l1-1-0.dll
 0000:fffd9000       .debug$S                   0000000180000000     ucrt:api-ms-win-crt-stdio-l1-1-0.dll
 0000:fffd9000       .debug$S                   0000000180000000     ucrt:api-ms-win-crt-string-l1-1-0.dll
 0000:fffd9000       .debug$S                   0000000180000000     ucrt:api-ms-win-crt-string-l1-1-0.dll
 0000:fffd9000       .debug$S                   0000000180000000     ucrt:api-ms-win-crt-string-l1-1-0.dll
 0000:fffd9000       .debug$S                   0000000180000000     ucrt:api-ms-win-crt-string-l1-1-0.dll
 0000:fffd9000       .debug$S                   0000000180000000     ucrt:api-ms-win-crt-string-l1-1-0.dll
 0000:fffd9000       .debug$S                   0000000180000000     ucrt:api-ms-win-crt-string-l1-1-0.dll
 0000:fffd9000       .debug$S                   0000000180000000     ucrt:api-ms-win-crt-string-l1-1-0.dll
 0000:fffd9000       .debug$S                   0000000180000000     ucrt:api-ms-win-crt-string-l1-1-0.dll
 0000:fffd9000       .debug$S                   0000000180000000     kernel32:KERNEL32.dll
 0000:fffd9000       .debug$S                   0000000180000000     kernel32:KERNEL32.dll
 0000:fffd9000       .debug$S                   0000000180000000     kernel32:KERNEL32.dll
 0000:fffd9000       .debug$S                   0000000180000000     kernel32:KERNEL32.dll
 0000:fffd9000       .debug$S                   0000000180000000     kernel32:KERNEL32.dll
 0000:fffd9000       .debug$S                   0000000180000000     kernel32:KERNEL32.dll
 0000:fffd9000       .debug$S                   0000000180000000     kernel32:KERNEL32.dll
 0000:fffd9000       .debug$S                   0000000180000000     kernel32:KERNEL32.dll
 0000:fffd9000       .debug$S                   0000000180000000     kernel32:KERNEL32.dll
 0000:fffd9000       .debug$S                   0000000180000000     kernel32:KERNEL32.dll
 0000:fffd9000       .debug$S                   0000000180000000     kernel32:KERNEL32.dll
 0000:fffd9000       .debug$S                   0000000180000000     kernel32:KERNEL32.dll
 0000:fffd9000       .debug$S                   0000000180000000     kernel32:KERNEL32.dll
 0000:fffd9000       .debug$S                   0000000180000000     kernel32:KERNEL32.dll
 0000:fffd9000       .debug$S                   0000000180000000     kernel32:KERNEL32.dll
 0000:fffd9000       .debug$S                   0000000180000000     kernel32:KERNEL32.dll
 0000:fffd9000       .debug$S                   0000000180000000     kernel32:KERNEL32.dll
 0000:fffd9000       .debug$S                   0000000180000000     kernel32:KERNEL32.dll
 0000:fffd9000       .debug$S                   0000000180000000     kernel32:KERNEL32.dll
 0000:fffd9000       .debug$S                   0000000180000000     kernel32:KERNEL32.dll
 0000:fffd9000       .debug$S                   0000000180000000     kernel32:KERNEL32.dll
 0000:fffd9000       .debug$S                   0000000180000000     kernel32:KERNEL32.dll
 0000:fffd9000       .debug$S                   0000000180000000     kernel32:KERNEL32.dll
 0000:fffd9000       .debug$S                   0000000180000000     kernel32:KERNEL32.dll
 0000:fffd9000       .debug$S                   0000000180000000     kernel32:KERNEL32.dll
 0000:fffd9000       .debug$S                   0000000180000000     kernel32:KERNEL32.dll
 0000:fffd9000       .debug$S                   0000000180000000     kernel32:KERNEL32.dll
 0000:fffd9000       .debug$S                   0000000180000000     kernel32:KERNEL32.dll
 0001:00000ee0       addRefToVerify             0000000180001ee0 f   libSetNativeMethodPrefix002.obj
 0001:00000f54       agentThreadWrapper         0000000180001f54 f   libSetNativeMethodPrefix002.obj
 0001:000010a8       check_option               00000001800020a8 f   libSetNativeMethodPrefix002.obj
 0001:000012f0       file_basename              00000001800022f0 f   libSetNativeMethodPrefix002.obj
 0001:00001dd8       startAgentThreadWrapper    0000000180002dd8 f   libSetNativeMethodPrefix002.obj
 0001:00002104       syncDebuggeeStatus         0000000180003104 f   libSetNativeMethodPrefix002.obj
 0001:0000238c       capture_previous_context   000000018000338c f   MSVCRT:gs_report.obj
 0001:00002400       ?__scrt_initialize_thread_safe_statics@@YAHXZ 0000000180003400 f   MSVCRT:thread_safe_statics.obj
 0001:000024d0       ?__scrt_uninitialize_thread_safe_statics@@YAXXZ 00000001800034d0 f   MSVCRT:thread_safe_statics.obj
 0001:00002580       $$000000                   0000000180003580     MSVCRT:amdsecgs.obj
 0001:000025b0       ?dllmain_crt_dispatch@@YAHQEAUHINSTANCE__@@KQEAX@Z 00000001800035b0 f   MSVCRT:dll_dllmain.obj
 0001:00002600       ?dllmain_crt_process_attach@@YAHQEAUHINSTANCE__@@QEAX@Z 0000000180003600 f   MSVCRT:dll_dllmain.obj
 0001:00002718       ?dllmain_crt_process_detach@@YAH_N@Z 0000000180003718 f   MSVCRT:dll_dllmain.obj
 0001:0000279c       ?dllmain_dispatch@@YAHQEAUHINSTANCE__@@KQEAX@Z 000000018000379c f   MSVCRT:dll_dllmain.obj
 0001:000031b0       $$000000                   00000001800041b0     MSVCRT:guard_dispatch.obj
 0001:000031d0       $$000000                   00000001800041d0     MSVCRT:guard_xfg_dispatch.obj
 0001:000031e6       ?fin$0@?0??dllmain_crt_process_attach@@YAHQEAUHINSTANCE__@@QEAX@Z@4HA 00000001800041e6 f   MSVCRT:dll_dllmain.obj
 0001:000031fd       ?fin$0@?0??dllmain_crt_process_detach@@YAH_N@Z@4HA 00000001800041fd f   MSVCRT:dll_dllmain.obj
 0001:00003216       ?fin$1@?0??dllmain_crt_process_detach@@YAH_N@Z@4HA 0000000180004216 f   MSVCRT:dll_dllmain.obj
 0001:0000322a       ?filt$0@?0??dllmain_dispatch@@YAHQEAUHINSTANCE__@@KQEAX@Z@4HA 000000018000422a f   MSVCRT:dll_dllmain.obj
 0001:00003260       __scrt_is_nonwritable_in_current_image$filt$0 0000000180004260 f   MSVCRT:utility.obj
 0002:00000218       ?__scrt_initialize_tss_var@@3P6AHXZEA 0000000180005218     MSVCRT:thread_safe_statics.obj
 0002:00000340       ?opcLengths@@3QBEB         0000000180005340     libSetNativeMethodPrefix002.obj
 0002:00001e80       GS_ExceptionPointers       0000000180006e80     MSVCRT:gs_report.obj
 0002:00002538       $unwind$fprintf            0000000180007538     libSetNativeMethodPrefix002.obj
 0002:00002544       $unwind$printf             0000000180007544     libSetNativeMethodPrefix002.obj
 0002:00002550       $unwind$?NewObject@JNIEnv_@@QEAAPEAV_jobject@@PEAV_jclass@@PEAU_jmethodID@@ZZ 0000000180007550     libSetNativeMethodPrefix002.obj
 0002:00002550       $unwind$nsk_lcomplain      0000000180007550     libSetNativeMethodPrefix002.obj
 0002:00002550       $unwind$nsk_ldisplay       0000000180007550     libSetNativeMethodPrefix002.obj
 0002:00002558       $unwind$nsk_lvdisplay      0000000180007558     libSetNativeMethodPrefix002.obj
 0002:00002558       $unwind$_RTC_Initialize    0000000180007558     MSVCRT:initsect.obj
 0002:00002558       $unwind$_RTC_Terminate     0000000180007558     MSVCRT:initsect.obj
 0002:00002558       $unwind$?__scrt_initialize_thread_safe_statics@@YAHXZ 0000000180007558     MSVCRT:thread_safe_statics.obj
 0002:00002564       $unwind$nsk_complain       0000000180007564     libSetNativeMethodPrefix002.obj
 0002:00002564       $unwind$nsk_printf         0000000180007564     libSetNativeMethodPrefix002.obj
 0002:0000256c       $unwind$nsk_lvcomplain     000000018000756c     libSetNativeMethodPrefix002.obj
 0002:00002584       $unwind$nsk_ltrace         0000000180007584     libSetNativeMethodPrefix002.obj
 0002:00002584       $unwind$__report_gsfailure 0000000180007584     MSVCRT:gs_report.obj
 0002:0000258c       $unwind$nsk_lvtrace        000000018000758c     libSetNativeMethodPrefix002.obj
 0002:0000258c       $unwind$__raise_securityfailure 000000018000758c     MSVCRT:gs_report.obj
 0002:0000258c       $unwind$__scrt_initialize_crt 000000018000758c     MSVCRT:utility.obj
 0002:0000258c       $unwind$__scrt_initialize_onexit_tables 000000018000758c     MSVCRT:utility.obj
 0002:0000258c       $unwind$__scrt_release_startup_lock 000000018000758c     MSVCRT:utility.obj
 0002:0000258c       $unwind$__scrt_uninitialize_crt 000000018000758c     MSVCRT:utility.obj
 0002:0000258c       $unwind$_onexit            000000018000758c     MSVCRT:utility.obj
 0002:00002594       $unwind$nsk_lverify        0000000180007594     libSetNativeMethodPrefix002.obj
 0002:000025a4       $unwind$nsk_vprintf        00000001800075a4     libSetNativeMethodPrefix002.obj
 0002:000025b4       $unwind$?nsk_jni_lverify@@YAHHPEAUJNIEnv_@@HQEBDH1ZZ 00000001800075b4     libSetNativeMethodPrefix002.obj
 0002:000025c8       $unwind$?nsk_jni_check_exception@@YAHPEAUJNIEnv_@@QEBDH@Z 00000001800075c8     libSetNativeMethodPrefix002.obj
 0002:000025e4       $unwind$nsk_jvmti_parseOptions 00000001800075e4     libSetNativeMethodPrefix002.obj
 0002:00002600       $unwind$nsk_jvmti_createJVMTIEnv 0000000180007600     libSetNativeMethodPrefix002.obj
 0002:00002614       $unwind$Java_nsk_jvmti_SetNativeMethodPrefix_SetNativeMethodPrefix002_foo 0000000180007614     libSetNativeMethodPrefix002.obj
 0002:00002614       $unwind$Java_nsk_jvmti_unit_FollowReferences_FollowRefObjects_resetTags 0000000180007614     libSetNativeMethodPrefix002.obj
 0002:00002614       $unwind$addRefToVerify     0000000180007614     libSetNativeMethodPrefix002.obj
 0002:00002614       $unwind$nsk_jvmti_resetAgentData 0000000180007614     libSetNativeMethodPrefix002.obj
 0002:00002614       $unwind$__scrt_initialize_default_local_stdio_options 0000000180007614     MSVCRT:default_local_stdio_options.obj
 0002:00002614       $unwind$?dllmain_crt_dispatch@@YAHQEAUHINSTANCE__@@KQEAX@Z 0000000180007614     MSVCRT:dll_dllmain.obj
 0002:00002614       $unwind$DllMain            0000000180007614     MSVCRT:dll_dllmain_stub.obj
 0002:00002614       $unwind$__GSHandlerCheck   0000000180007614     MSVCRT:gshandler.obj
 0002:00002614       $unwind$?__scrt_uninitialize_thread_safe_statics@@YAXXZ 0000000180007614     MSVCRT:thread_safe_statics.obj
 0002:00002614       $unwind$__scrt_acquire_startup_lock 0000000180007614     MSVCRT:utility.obj
 0002:00002614       $unwind$__scrt_dllmain_after_initialize_c 0000000180007614     MSVCRT:utility.obj
 0002:00002614       $unwind$__scrt_dllmain_before_initialize_c 0000000180007614     MSVCRT:utility.obj
 0002:00002614       $unwind$__scrt_dllmain_crt_thread_attach 0000000180007614     MSVCRT:utility.obj
 0002:00002614       $unwind$__scrt_dllmain_crt_thread_detach 0000000180007614     MSVCRT:utility.obj
 0002:00002614       $unwind$__scrt_dllmain_uninitialize_c 0000000180007614     MSVCRT:utility.obj
 0002:00002614       $unwind$__scrt_dllmain_uninitialize_critical 0000000180007614     MSVCRT:utility.obj
 0002:00002614       $unwind$atexit             0000000180007614     MSVCRT:utility.obj
 0002:0000261c       $unwind$check_option       000000018000761c     libSetNativeMethodPrefix002.obj
 0002:0000261c       $unwind$nsk_jvmti_findOptionValue 000000018000761c     libSetNativeMethodPrefix002.obj
 0002:0000261c       $unwind$_DllMainCRTStartup 000000018000761c     MSVCRT:dll_dllmain.obj
 0002:0000262c       $unwind$nsk_jvmti_findOptionIntValue 000000018000762c     libSetNativeMethodPrefix002.obj
 0002:0000263c       $unwind$nsk_jvmti_lverify  000000018000763c     libSetNativeMethodPrefix002.obj
 0002:00002650       $unwind$exitOnError        0000000180007650     libSetNativeMethodPrefix002.obj
 0002:00002660       $unwind$Java_nsk_share_jvmti_ArgumentHandler_getAgentOptionsString 0000000180007660     libSetNativeMethodPrefix002.obj
 0002:00002674       $unwind$Java_nsk_jvmti_unit_FollowReferences_FollowRefObjects_getTag 0000000180007674     libSetNativeMethodPrefix002.obj
 0002:00002674       $unwind$Java_nsk_share_jvmti_DebugeeClass_checkStatus 0000000180007674     libSetNativeMethodPrefix002.obj
 0002:00002674       $unwind$agentThreadWrapper 0000000180007674     libSetNativeMethodPrefix002.obj
 0002:00002684       $unwind$startAgentThreadWrapper 0000000180007684     libSetNativeMethodPrefix002.obj
 0002:000026a0       $unwind$syncDebuggeeStatus 00000001800076a0     libSetNativeMethodPrefix002.obj
 0002:000026a0       $unwind$__scrt_dllmain_exception_filter 00000001800076a0     MSVCRT:utility.obj
 0002:000026b4       $unwind$Java_nsk_share_jvmti_DebugeeClass_resetAgentData 00000001800076b4     libSetNativeMethodPrefix002.obj
 0002:000026bc       $unwind$MA_checkStatus     00000001800076bc     libSetNativeMethodPrefix002.obj
 0002:000026d0       $unwind$Java_nsk_jvmti_unit_FollowReferences_FollowRefObjects_setTag 00000001800076d0     libSetNativeMethodPrefix002.obj
 0002:000026e8       $unwind$Java_nsk_jvmti_unit_FollowReferences_FollowRefObjects_addRefToVerify 00000001800076e8     libSetNativeMethodPrefix002.obj
 0002:00002704       $unwind$Agent_Initialize   0000000180007704     libSetNativeMethodPrefix002.obj
 0002:00002720       $unwind$capture_previous_context 0000000180007720     MSVCRT:gs_report.obj
 0002:0000272c       $unwind$__GSHandlerCheckCommon 000000018000772c     MSVCRT:gshandler.obj
 0002:00002738       $xdatasym                  0000000180007738     MSVCRT:amdsecgs.obj
 0002:0000273c       $unwind$?dllmain_crt_process_attach@@YAHQEAUHINSTANCE__@@QEAX@Z 000000018000773c     MSVCRT:dll_dllmain.obj
 0002:00002778       $unwind$?fin$0@?0??dllmain_crt_process_attach@@YAHQEAUHINSTANCE__@@QEAX@Z@4HA 0000000180007778     MSVCRT:dll_dllmain.obj
 0002:00002778       $unwind$?fin$0@?0??dllmain_crt_process_detach@@YAH_N@Z@4HA 0000000180007778     MSVCRT:dll_dllmain.obj
 0002:00002778       $unwind$?fin$1@?0??dllmain_crt_process_detach@@YAH_N@Z@4HA 0000000180007778     MSVCRT:dll_dllmain.obj
 0002:00002780       $unwind$?dllmain_crt_process_detach@@YAH_N@Z 0000000180007780     MSVCRT:dll_dllmain.obj
 0002:000027d4       $unwind$?dllmain_dispatch@@YAHQEAUHINSTANCE__@@KQEAX@Z 00000001800077d4     MSVCRT:dll_dllmain.obj
 0002:000027fc       $unwind$?filt$0@?0??dllmain_dispatch@@YAHQEAUHINSTANCE__@@KQEAX@Z@4HA 00000001800077fc     MSVCRT:dll_dllmain.obj
 0002:00002804       $unwind$__scrt_is_nonwritable_in_current_image 0000000180007804     MSVCRT:utility.obj
 0002:00002824       $unwind$__scrt_is_nonwritable_in_current_image$filt$0 0000000180007824     MSVCRT:utility.obj
 0002:0000282c       $unwind$__scrt_fastfail    000000018000782c     MSVCRT:utility_desktop.obj
 0002:0000283c       $unwind$__security_init_cookie 000000018000783c     MSVCRT:gs_support.obj
 0002:00002848       $unwind$__isa_available_init 0000000180007848     MSVCRT:cpu_disp.obj
 0002:00002858       $xdatasym                  0000000180007858     MSVCRT:guard_dispatch.obj
 0002:00002860       $xdatasym                  0000000180007860     MSVCRT:guard_xfg_dispatch.obj
 0002:00002870       .edata                     0000000180007870     SetNativeMethodPrefix002.exp
 0002:00002898       rgpv                       0000000180007898     SetNativeMethodPrefix002.exp
 0002:000028d4       rgszName                   00000001800078d4     SetNativeMethodPrefix002.exp
 0002:00002910       rgwOrd                     0000000180007910     SetNativeMethodPrefix002.exp
 0002:0000292e       szName                     000000018000792e     SetNativeMethodPrefix002.exp
 0002:0000294b       $N00001                    000000018000794b     SetNativeMethodPrefix002.exp
 0002:0000295a       $N00002                    000000018000795a     SetNativeMethodPrefix002.exp
 0002:00002967       $N00003                    0000000180007967     SetNativeMethodPrefix002.exp
 0002:000029a9       $N00004                    00000001800079a9     SetNativeMethodPrefix002.exp
 0002:000029ee       $N00005                    00000001800079ee     SetNativeMethodPrefix002.exp
 0002:00002a2b       $N00006                    0000000180007a2b     SetNativeMethodPrefix002.exp
 0002:00002a73       $N00007                    0000000180007a73     SetNativeMethodPrefix002.exp
 0002:00002ab3       $N00008                    0000000180007ab3     SetNativeMethodPrefix002.exp
 0002:00002af0       $N00009                    0000000180007af0     SetNativeMethodPrefix002.exp
 0002:00002b2b       $N00010                    0000000180007b2b     SetNativeMethodPrefix002.exp
 0002:00002b59       $N00011                    0000000180007b59     SetNativeMethodPrefix002.exp
 0002:00002b8a       $N00012                    0000000180007b8a     SetNativeMethodPrefix002.exp
 0002:00002bb9       $N00013                    0000000180007bb9     SetNativeMethodPrefix002.exp
 0002:00002be8       $N00014                    0000000180007be8     SetNativeMethodPrefix002.exp
 0002:00002c1d       $N00015                    0000000180007c1d     SetNativeMethodPrefix002.exp
 0002:00003082       .idata$6                   0000000180008082     kernel32:KERNEL32.dll
 0002:000030e6       .idata$6                   00000001800080e6     vcruntime:VCRUNTIME140.dll
 0002:00003278       .idata$6                   0000000180008278     ucrt:api-ms-win-crt-heap-l1-1-0.dll
 0002:00003298       .idata$6                   0000000180008298     ucrt:api-ms-win-crt-runtime-l1-1-0.dll
 0002:000032ba       .idata$6                   00000001800082ba     ucrt:api-ms-win-crt-convert-l1-1-0.dll
 0002:000032dc       .idata$6                   00000001800082dc     ucrt:api-ms-win-crt-stdio-l1-1-0.dll
 0002:000032fc       .idata$6                   00000001800082fc     ucrt:api-ms-win-crt-string-l1-1-0.dll
 0003:00000000       ?codeAttributeName@@3PEBDEB 0000000180009000     libSetNativeMethodPrefix002.obj
 0003:00000008       ?lineNumberAttributeName@@3PEBDEB 0000000180009008     libSetNativeMethodPrefix002.obj
 0003:00000010       ?localVarAttributeName@@3PEBDEB 0000000180009010     libSetNativeMethodPrefix002.obj
 0003:00000018       ?localVarTypeAttributeName@@3PEBDEB 0000000180009018     libSetNativeMethodPrefix002.obj
 0003:00000020       ?stackMapAttributeName@@3PEBDEB 0000000180009020     libSetNativeMethodPrefix002.obj
 0003:00000028       ?callBytes@@3PAEA          0000000180009028     libSetNativeMethodPrefix002.obj
 0003:0000002c       ?allocBytes@@3PAEA         000000018000902c     libSetNativeMethodPrefix002.obj
 0003:0001aad4       redefineAttempted          0000000180023ad4     libSetNativeMethodPrefix002.obj
 0003:0001aad8       nsk_context                0000000180023ad8     libSetNativeMethodPrefix002.obj
 0003:0001aae4       redefineSucceed            0000000180023ae4     libSetNativeMethodPrefix002.obj
 0003:0001aae8       agentFailed                0000000180023ae8     libSetNativeMethodPrefix002.obj
 0003:0001aaec       currentAgentStatus         0000000180023aec     libSetNativeMethodPrefix002.obj
 0003:0001aaf0       context                    0000000180023af0     libSetNativeMethodPrefix002.obj
 0003:0001aba8       agentThread                0000000180023ba8     libSetNativeMethodPrefix002.obj
 0003:0001abb0       agentThreadProc            0000000180023bb0     libSetNativeMethodPrefix002.obj
 0003:0001abb8       agentThreadArg             0000000180023bb8     libSetNativeMethodPrefix002.obj
 0003:0001abc0       agent_data                 0000000180023bc0     libSetNativeMethodPrefix002.obj
 0003:0001abd0       jvmti_env                  0000000180023bd0     libSetNativeMethodPrefix002.obj
 0003:0001abd8       jvm                        0000000180023bd8     libSetNativeMethodPrefix002.obj
 0003:0001abe0       jni_env                    0000000180023be0     libSetNativeMethodPrefix002.obj
 0003:0001abe8       checkStatus_func           0000000180023be8     libSetNativeMethodPrefix002.obj
 0003:0001abf0       ?codeAttributeIndex@@3GA   0000000180023bf0     libSetNativeMethodPrefix002.obj
 0003:0001abf4       ?lineNumberAttributeIndex@@3GA 0000000180023bf4     libSetNativeMethodPrefix002.obj
 0003:0001abf8       ?localVarAttributeIndex@@3GA 0000000180023bf8     libSetNativeMethodPrefix002.obj
 0003:0001abfc       ?localVarTypeAttributeIndex@@3GA 0000000180023bfc     libSetNativeMethodPrefix002.obj
 0003:0001ac00       ?stackMapAttributeIndex@@3GA 0000000180023c00     libSetNativeMethodPrefix002.obj
 0003:0001ac04       ?stackFrameOffset@@3GA     0000000180023c04     libSetNativeMethodPrefix002.obj
 0003:0001ac08       ?mode@@3HA                 0000000180023c08     libSetNativeMethodPrefix002.obj
 0003:0001ac0c       ?constantPoolSize@@3GA     0000000180023c0c     libSetNativeMethodPrefix002.obj
 0003:0001ac10       ?orig@@3PEBEEB             0000000180023c10     libSetNativeMethodPrefix002.obj
 0003:0001ac18       ?gen@@3PEAEEA              0000000180023c18     libSetNativeMethodPrefix002.obj
 0003:0001ac20       ?inputPos@@3PEAEEA         0000000180023c20     libSetNativeMethodPrefix002.obj
 0003:0001ac28       ?endPos@@3PEBEEB           0000000180023c28     libSetNativeMethodPrefix002.obj
 0003:0001ac30       ?genPos@@3PEAEEA           0000000180023c30     libSetNativeMethodPrefix002.obj
 0003:0001ac38       ?markPos@@3PEAEEA          0000000180023c38     libSetNativeMethodPrefix002.obj
 0003:0001ac40       ?constantPool@@3PEAPEADEA  0000000180023c40     libSetNativeMethodPrefix002.obj
 0003:0001ac48       ?constantPoolCount@@3GA    0000000180023c48     libSetNativeMethodPrefix002.obj
 0003:0001ac4c       ?zeroBytes@@3PAEA          0000000180023c4c     libSetNativeMethodPrefix002.obj
 0003:0001ac50       ?codeLength@@3IA           0000000180023c50     libSetNativeMethodPrefix002.obj
 0003:0001ac58       ?map@@3PEAIEA              0000000180023c58     libSetNativeMethodPrefix002.obj
 0003:0001ac60       ?widening@@3PEACEA         0000000180023c60     libSetNativeMethodPrefix002.obj
 0003:0001ac68       prefix                     0000000180023c68     libSetNativeMethodPrefix002.obj
 0003:0001ac70       jvmti                      0000000180023c70     libSetNativeMethodPrefix002.obj
 0003:0001ac80       GS_ExceptionRecord         0000000180023c80     MSVCRT:gs_report.obj
 0003:0001ad20       GS_ContextRecord           0000000180023d20     MSVCRT:gs_report.obj
 0003:0001b1f0       ?g_tss_cv@@3U_RTL_CONDITION_VARIABLE@@A 00000001800241f0     MSVCRT:thread_safe_statics.obj
 0003:0001b1f8       ?g_tss_event@@3PEAXEA      00000001800241f8     MSVCRT:thread_safe_statics.obj
 0003:0001b200       ?g_tss_mutex@@3U_RTL_CRITICAL_SECTION@@A 0000000180024200     MSVCRT:thread_safe_statics.obj
 0003:0001b228       ?g_sleep_condition_variable_cs@@3P6AHPEAU_RTL_CONDITION_VARIABLE@@PEAU_RTL_CRITICAL_SECTION@@K@ZEA 0000000180024228     MSVCRT:thread_safe_statics.obj
 0003:0001b230       ?g_wake_all_condition_variable@@3P6AXPEAU_RTL_CONDITION_VARIABLE@@@ZEA 0000000180024230     MSVCRT:thread_safe_statics.obj
 0003:0001b23c       ?__proc_attached@@3HA      000000018002423c     MSVCRT:dll_dllmain.obj
 0003:0001b250       ?is_initialized_as_dll@@3_NA 0000000180024250     MSVCRT:utility.obj
 0003:0001b251       ?module_local_atexit_table_initialized@@3_NA 0000000180024251     MSVCRT:utility.obj
 0003:0001b258       ?module_local_atexit_table@@3U_onexit_table_t@@A 0000000180024258     MSVCRT:utility.obj
 0003:0001b270       ?module_local_at_quick_exit_table@@3U_onexit_table_t@@A 0000000180024270     MSVCRT:utility.obj
